:020000040800F2
:1000000000040020E1010008E3010008E30100080A
:10001000E3010008E3010008E3010008E301000830
:10002000E3010008E3010008E30100086527000878
:10003000E3010008E3010008E3010008E301000810
:10004000E3010008E3010008E3010008E301000800
:10005000E3010008E3010008CD380008F938000882
:1000600025390008513900087D390008E3010008EE
:10007000E3010008E3010008E3010008E3010008D0
:10008000E3010008E3010008E3010008E3010008C0
:10009000E3010008E3010008E3010008A9390008B2
:1000A000E3010008E3010008E3010008E3010008A0
:1000B000E3010008E3010008E3010008E301000890
:1000C000E3010008E3010008E3010008E301000880
:1000D000E3010008E30100088510000899100008FA
:1000E000113A0008E3010008E3010008E3010008F9
:1000F000E3010008E3010008E3010008E301000850
:10010000E3010008E3010008DD360008E301000810
:10011000E3010008E3010008E3010008E30100082F
:10012000E3010008E3010008E3010008E30100081F
:10013000E3010008E3010008E3010008E30100080F
:10014000E3010008E3010008E3010008512E000864
:10015000E3010008E3010008E3010008E3010008EF
:10016000E3010008E3010008E3010008E3010008DF
:10017000E3010008E3010008E3010008E3010008CF
:10018000E3010008E3010008AD100008E3010008E6
:10019000E3010008E3010008E3010008E3010008AF
:1001A000E3010008E3010008E3010008E30100089F
:1001B000E3010008E3010008E3010008E30100088F
:1001C000E3010008E3010008E3010008E30100087F
:1001D000E3010008E3010008E3010008E30100086F
:1001E00002E000F000F8FEE772B6394880F30888B4
:1001F000384880F3098838484EF60851CEF200019D
:10020000086040F20000CCF200004EF63471CEF2ED
:1002100000010860BFF34F8FBFF36F8F40F2000003
:10022000C0F2F0004EF68851CEF200010860BFF334
:100230004F8FBFF36F8F4FF00000E1EE100A4EF6C4
:100240003C71CEF200010860062080F31488BFF3F1
:100250006F8F02F0C5FA03F0D7F94FF055301F4900
:100260001B4A91423CBF41F8040BFAE71C49194A6A
:1002700091423CBF41F8040BFAE71A491A4A1B4B5A
:100280009A423EBF51F8040B42F8040BF8E70020F5
:100290001749184A91423CBF41F8040BFAE702F0B3
:1002A000A3FA03F00DFA144C144DAC4203DA54F8DF
:1002B000041B8847F9E700F03FF8114C114DAC42A0
:1002C00003DA54F8041B8847F9E702F08BBA000000
:1002D000000400200024002000000008000000208E
:1002E00000040020D03E0008002400202824002024
:1002F0002824002090410020E0010008E0010008CF
:10030000E0010008E00100082DE9F04F2DED108A12
:10031000C1F80CD0C3689D46BDEC108ABDE8F08FD3
:10032000002383F311882846A047002001F09CFE9B
:1003300001F04CFE00DFFEE770B5214C6FF01403B6
:1003400023700323002563706FF03F061F23A57001
:10035000E57025716571A571E57125726672A372EC
:10036000E57200F00DFD20B10F2325726672A372B5
:10037000E57202F0CDF9044602F0EEF90546D8B96F
:10038000104B9C421AD001339C4218BF054641F2E3
:10039000883404BF01250024002002F0C3F90DB108
:1003A00000F0B6F800F070FD00F028FC204600F0E8
:1003B0000DF900F0ADF8F9E70024EDE70446EBE7AE
:1003C00028240020010007B008B500F095FBA0F13B
:1003D00020035842584108BD07B5054B02211B8830
:1003E000ADF8043001A800F0F3FB03B05DF804FBA6
:1003F000103B0008064991F8243033B1002308224D
:10040000086A81F8243000F01BBC0120704700BF4F
:10041000482400202DE9F84F234C94F82430054659
:10042000884617468BBB2E46DFF87C90002F38D0CD
:1004300094F824A0BAF1000F05D12022FF214846EC
:10044000266200F00FFDCAF10805BD4228BF3D46F7
:100450005FFA85FBAD0041462A4604EB8A0000F0B6
:10046000D7FC94F82430A7EB0B079B445FFA8BFB77
:10047000BBF1080F2E44A844FFB284F824B0D5D1B4
:10048000FFF7B8FF0028D1D108E0266A06EB830603
:10049000B042C9D0FFF7AEFF0028C4D10020BDE8AC
:1004A000F88F0120BDE8F88F4824002010B52023E4
:1004B00083F311881248C3680BB101F05BFE00237F
:1004C000104A0F484FF47A7101F018FE002383F3AD
:1004D00011880D4C236813B12368013B23606368C6
:1004E00013B16368013B6360084B1B7833B96368E1
:1004F00023B9022000F082FC3223636010BD00BFEC
:1005000034240020AD040008782900207024002045
:1005100010B5254B254953F8042F013200D110BDE9
:100520008B42F8D1224C234B22689A423AD9224B73
:100530009B6803F1006303F580439A4232D20020A6
:1005400000F076FB1D4B0220187000F04DFC1C4B98
:100550001A6C00221A64196E1A66196E596C5A6464
:10056000596E5A665A6E5A6942F080025A615A6947
:1005700022F080025A615A691A6942F000521A61E7
:100580001A6922F000521A611B6972B60D4A0E4BAD
:1005900013601B682268202181F311889D4683F334
:1005A0000888104710BD00BFFC3F00081C40000831
:1005B00004400008FF3F0008282400207024002089
:1005C0000038024008ED00E0004000082DE9F04F3F
:1005D000B04C97B020228146FF210EA8A66800F0FB
:1005E00041FCAD4A1378A346A3B9AC480121C360CE
:1005F0001170202383F31188C3680BB101F0BAFD99
:100600000023A74AA5484FF47A7101F077FD002333
:1006100083F31188B9F1000F02D0A24BC3F8009008
:10062000A14BA04A00241C705460254627469846DA
:10063000012000F0D9FBB9F1000F00F02282994BA4
:100640001B68002B40F01D8217B0BDE8F08F022020
:10065000FFF7BAFE002840F00E82944B1B88ADF8DD
:100660002430022109A800F0B3FAE1E74FF47A70D0
:1006700000F042FA031E0193EFDB0220FFF7A4FE15
:1006800082460028E9D0019B581E042800F2F5811B
:10069000DFE800F0030D1013160016A8052340F83C
:1006A000343D042100F094FA5446002752E004211E
:1006B0007848F7E704217E48F4E704217D48F1E714
:1006C0001C24204600F0B6FA04340990042109A83D
:1006D00000F07EFA2C2CF4D1E6E7002DBDD0002CE2
:1006E000BBD00220FFF770FE0546002800F0C7814E
:1006F000012000F09DFA022088F8000000F074FB51
:100700000024E3B21846019300F0A2FA824648B1F1
:10071000019B184600F0ACFA01340028F1D12C46B8
:10072000654B9BE70123022088F8003000F052FB64
:100730005646DBF808309E4206D2304600F07AFA80
:100740000130ECD10436F4E7564B002688F80060FF
:100750005E602C4600F08EFB1DB1002C18BF4FF0E0
:100760000009FFF739FE63E7002D3FF476AF002C58
:100770003FF473AF022088F8000000F035FB322010
:1007800000F0BAF9B0F1000AC0F279811AF003055D
:1007900040F07581DBF8082006EB0A03934200F273
:1007A0006E81BAF5807F00F26A81444B0193554512
:1007B0000DDA4FF47A7000F09FF90290029A002A45
:1007C000C0F25D81019B029AEA540135EEE7C82030
:1007D000FFF7FAFD0546002800F051811F2E11D8C1
:1007E000C6F12004544528BF54460EAB26F0030042
:1007F00022463249184400F00BFB2246FF212F48C5
:1008000000F030FB4FEAAA0A5FFA8AF22B49304621
:10081000FFF700FE0446002881D006EB8A06054655
:1008200098E70220FFF7D0FD00283FF416AFFFF74E
:10083000E1FD00283FF411AF00229246DBF80830BA
:100840009A4259D21F2A1ED80E9B01331BD022F088
:10085000030316A90B4453F8203C09931848436836
:1008600083B3174800210DF1240E11F80E3083EAEE
:100870000A03DBB2013150F82330042983EA1A2A33
:10088000F3D10432DAE71046019200F0D3F9019A6D
:100890000990E3E728240020742500203424002058
:1008A000AD0400087829002070240020123B0008C5
:1008B0002C24002030240020143B00087424002045
:1008C0007825002019464FF0080E11F0010F4FEA6D
:1008D00051011FBF81F06D4181F4380181F4034162
:1008E00081F02001BEF1010EEFD140F82310013359
:1008F000B3F5807FE6D1B4E716A8042140F84CADEB
:1009000000F066F926E716A8002340F8343D64217C
:1009100000F02AF900287FF4A0AE0220FFF754FD72
:1009200000283FF49AAE099800F0B4F916AB43F8EA
:10093000480D04211846E3E716A8002340F8343D8B
:10094000642100F011F900287FF487AE0220FFF740
:100950003BFD00283FF481AE099800F0A9F916ABE1
:1009600043F8440DE5E70220FFF72EFD00283FF491
:1009700074AE00F0A3F916AB43F8400DD9E702209E
:10098000FFF722FD00283FF468AE09A9142000F00B
:100990009BF9824616A8042140F83CAD00F018F9F6
:1009A000514609A8ACE7322000F0A6F8B0F1000AE1
:1009B000FFF653AE1AF0030F7FF44FAEDBF80820BA
:1009C0000AEB070393423FF648AE0220FFF7FCFC18
:1009D00000283FF442AE2AF0030ABA44BA453FF475
:1009E000B9AE384600F026F90421089008A800F0B6
:1009F000EFF80437F2E74FF47A70FFF7E5FC0028D0
:100A00003FF42BAEFFF7F6FC00283FF489AE0E9BB7
:100A100001330CD008220EA90020FFF7FBFC0028B0
:100A20003FF47EAE2022FF210EA800F01BFAFFF754
:100A3000D3FC304801F01EFB06E616A8002340F860
:100A4000343D642100F090F8824600287FF405AE22
:100A50000220FFF7B9FC00283FF4FFADFFF7BCFC14
:100A600041F2883001F006FB099800F047FAD146C0
:100A700000F000FADCE505466CE60027EDE52546CA
:100A8000EBE5002000F038F80290029B002BFFF607
:100A9000D2AD012000F09EF9029B213B122B3FF6C4
:100AA000C7AD01A252F823F04F0600086D060008FA
:100AB000DB06000831060008310600083106000890
:100AC00069070008A70900082308000807090008AB
:100AD0003909000867090008310600087F09000885
:100AE00031060008F709000855070008310600081C
:100AF0003B0A0008A08601002DE9F34702AE00245E
:100B00004FF47A7506F8014D144FDFF858804543CD
:100B100097F900305A1C5FFA84F901D0A34212D130
:100B200058F8240003680122D3F820A031462B4650
:100B3000D047012807D10A4B9DF8070083F80090A1
:100B400002B0BDE8F0870134042CE1D14FF4FA7013
:100B500001F090FA4FF0FF30F2E700BF00240020D0
:100B600098290020683B00082DE9F0474FF47A757A
:100B7000144FDFF8588006464D43002497F90030A3
:100B80005A1C5FFA84F901D0A34210D158F824000E
:100B900003680422D3F820A031462B46D04704280E
:100BA00005D1094B83F800900020BDE8F08701349F
:100BB000042CE3D14FF4FA7001F05CFA4FF0FF30EF
:100BC000BDE8F0870024002098290020683B000839
:100BD00030B4074B1A78074B53F822402368DD697D
:100BE000054B0A46AC460146204630BC604700BF74
:100BF00098290020683B0008A086010070B501F02C
:100C000083FC094C094E207000253068237883420C
:100C100008D901F073FC336805440133B5F5804F02
:100C20003360F2D370BD00BF9929002080290020D5
:100C300001F020BD00F1006000F5804000687047C1
:100C400000F10060920000F5804001F0ABBC0000B4
:100C5000054B1A68054B1B789B1A834202D9104436
:100C600001F04CBC00207047802900209929002009
:100C700038B5074D04462868204401F047FC28B9E0
:100C800028682044BDE8384001F058BC38BD00BF9A
:100C90008029002010F0030308D1B0F5007F05D8AB
:100CA00000F10050A0F50840006870470020704730
:100CB000014BC058704700BF107AFF1F014B1868E6
:100CC000704700BF002004E070B52A4B1C68C4F3D5
:100CD0000B03240C63B140F21342934231D040F233
:100CE000194293422FD040F2214293422DD1032347
:100CF000214A0C2505FB03235D6893F9082042F285
:100D000001039C4224D0B4F5805F23D041F201035B
:100D10009C4221D041F203039C421FD041F20703C1
:100D20009C4208BF3122441E0C44013D0B46A342A5
:100D30001ED215F9016F581C96B1034600F8016CDC
:100D4000F5E70123D4E70223D2E73F220B4DD6E794
:100D50003322E3E74122E1E75A22E4E75922E2E7BE
:100D60002C2584421D7001D9981C5A70401A70BD00
:100D70001846FBE7002004E0383B0008183B000859
:100D8000124B5A8842F201018A4293B214D0B3F551
:100D9000805F13D041F20102934211D041F203026D
:100DA00093420FD041F2070293420DD10423084A27
:100DB00002EB8303D87870470023F8E70123F6E7B6
:100DC0000223F4E70323F2E700207047002004E049
:100DD000243B0008022802BF024B4FF480529A6164
:100DE000704700BF00100240022802BF024B4FF0C4
:100DF00080529A61704700BF00100240022801BF74
:100E0000024A536983F480535361704700100240D3
:100E100010B50023934203D0CC5CC4540133F9E7EE
:100E200010BD000030B5441E14F9010F0B4660B12F
:100E300093F90050854201F1010106D11AB993F9E5
:100E40000020801A30BD013AEEE7002AF7D11046A3
:100E500030BD000002460346981A13F9011B002911
:100E6000FAD1704702440346934202D003F8011BB3
:100E7000FAE77047024B1A78024B1A70704700BFAE
:100E80009829002000240020F8B5164C1648174D6C
:100E9000174E154F00F036FC2146134800F05EFC5B
:100EA00024681448626D936B23F40023936301F06C
:100EB000E1F82046104900F05DFD626D936B43F44C
:100EC000002393634FF4E1332B60002456F8240091
:100ED000B84202D0294600F073FB0134042CF5D14E
:100EE000F8BD00BF503C00081437002084290020C2
:100EF000683B000840420F007C3C000838B50B4BB3
:100F00001A780B4B53F822400A4B9C4205460CD0F2
:100F1000094B002118461422FFF7A4FF0560014683
:100F20002046BDE8384000F04BBB38BD9829002072
:100F3000683B0008143700208429002002684368B9
:100F40001143016003B1184770470000024AD3689B
:100F500043F0C003D360704700440040024AD368A6
:100F600043F0C003D360704700480040024AD36892
:100F700043F0C003D3607047007800402DE9F04192
:100F8000D0F85C64F7683368DA0505469CB20DD585
:100F9000202383F311884FF400710430FFF7CEFF54
:100FA0006FF480733360002383F31188202383F36D
:100FB000118805F1040814F02F0333D183F311884D
:100FC000380615D5210613D5202383F3118805F1A2
:100FD000380000F053FA002846DA0821281DFFF7F0
:100FE000ADFF4FF67F733B40F360002383F311881E
:100FF0007A060ED563060CD5202383F31188EA6C9C
:101000002B6D9A4202D12B6C002B2FD1002383F33E
:101010001188D5F86424D368002B31D01069BDE85D
:10102000F0411847230713D014F0080F0CBF00211C
:101030008021E00748BF41F02001A20748BF41F0EE
:101040004001630748BF41F480714046FFF776FFD7
:10105000A406736805D595F860142846194000F079
:10106000BDFA3468A4B2A6E77060BEE727F0400777
:101070003F041021281D3F0CFFF760FFF760C5E714
:10108000BDE8F08108B50348FFF778FFBDE80840E8
:1010900001F078BB9C29002008B50348FFF76EFFDC
:1010A000BDE8084001F06EBB042E002008B50348DF
:1010B000FFF764FFBDE8084001F064BB6C3200201C
:1010C00010B50E4C0E4A2046002100F057FA0D4B89
:1010D000C4F85C340C4C0D4A2046002100F04EFA56
:1010E0000B4BC4F85C340B4C0B4A0021204600F03B
:1010F00045FA0A4BC4F85C3410BD00BF9C2900209F
:101100004D0F000800440040042E00205D0F000831
:10111000004800406C3200206D0F0008007800404D
:1011200038B5394D037C002918BF0D46012B044604
:10113000C0F8645410D1354B984242D1344B1A6CEC
:1011400042F400321A641A6E42F400321A661B6EC0
:101150000B21262000F06AF82E4BD4F85C249A422A
:101160002B6802D02C498A424BD12C4901EB530108
:10117000B1FBF3F3A988080442BF23F0070003F092
:10118000070343EA40039360EB8843F040039BB2BC
:1011900013612B8943F001039BB2536141F4045363
:1011A00043F02C03D36001F4A05100231360B1F588
:1011B000806F136853680CBF7F23FF2384F860346B
:1011C00038BD174B98420CD1114B1A6C42F4802257
:1011D0001A641A6E42F480221A661B6E0B212720B5
:1011E000B8E7104B9842B7D1094B1A6C42F08042D5
:1011F0001A641A6E42F080421A661B6E0B2152204E
:10120000A8E70949B2E700BF983B00089C290020E5
:1012100000380240001001400014014000BD0105EB
:10122000042E00206C32002080DE800200F160433A
:1012300000F01F02400903F5614309018000C9B2B3
:1012400000F1604083F8001300F5614001239340F2
:10125000C0F8803103607047F8B5154682680669AA
:10126000AA420B46816938BF8568761AB5420446A2
:1012700007D218462A46FFF7CBFDA3692B44A3618A
:101280000DE011D932461846FFF7C2FDAF1B3A46B2
:10129000E1683044FFF7BCFDE2683A44A261A3680C
:1012A0005B1BA3602846F8BD18462A46FFF7B0FD31
:1012B000E368E4E783682DE9F0410446934215466C
:1012C000266938BF85684069361AB5420F4606D28E
:1012D0002A46FFF79DFD63692B4463610DE012D937
:1012E0003246A5EB0608FFF793FD4246B919E068C0
:1012F000FFF78EFDE26842446261A3685B1BA36056
:101300002846BDE8F0812A46FFF782FDE368E4E75E
:1013100010B50A440024C361029B006040608460F1
:10132000C160816141610261036210BD08B58269DB
:101330004369934201D1826882B982680132826036
:101340005A1C42611970426903699A4201D3C36809
:101350004361002100F0AAFE002008BD4FF0FF30DD
:1013600008BD000070B5202304460E4683F31188A3
:10137000A568A5B1A368A269013BA360531CA36142
:1013800015782269934224BFE368A361E3690BB136
:1013900020469847002383F31188284670BD3146C4
:1013A000204600F073FE0028E2DA85F3118870BD54
:1013B0002DE9F74F05460F4690469A46D0F81C9007
:1013C000202686F311884FF0000B144664B12246A4
:1013D00039462846FFF740FF034668B9514628467C
:1013E00000F054FE0028F1D0002383F31188A8EB0D
:1013F000040003B0BDE8F08FB9F1000F03D00190F5
:101400002846C847019B8BF31188E41A1F4486F3D2
:101410001188DBE7C16081614161C3611144009BB8
:10142000006040608260016103627047F8B5044665
:101430000E461746202383F31188A568A5B1A3683B
:10144000013BA36063695A1C62611E702369626973
:101450009A4224BFE3686361E3690BB12046984771
:10146000002080F31188F8BD3946204600F00EFEBA
:101470000028E2DA85F31188F8BD0000836942692B
:101480009A4210B501D182687AB9826801328260CD
:101490005A1C82611C7803699A4201D3C368836134
:1014A000002100F003FE204610BD4FF0FF3010BDBC
:1014B0002DE9F74F05460F4690469A46D0F81C9006
:1014C000202686F311884FF0000B144664B12246A3
:1014D00039462846FFF7EEFE034668B951462846CE
:1014E00000F0D4FD0028F1D0002383F31188A8EB8D
:1014F000040003B0BDE8F08FB9F1000F03D00190F4
:101500002846C847019B8BF31188E41A1F4486F3D1
:101510001188DBE7026843681143016003B1184793
:10152000704700001430FFF743BF00004FF0FF3357
:101530001430FFF73DBF00003830FFF7B9BF00009F
:101540004FF0FF333830FFF7B3BF00001430FFF720
:1015500009BF00004FF0FF311430FFF703BF000058
:101560003830FFF763BF00004FF0FF323830FFF72D
:101570005DBF000000207047FFF7A2BD37B50F4BDD
:101580000360002343608360C36001230446037447
:10159000154600900B464FF4007200F15C011430C8
:1015A000FFF7B6FE00942B464FF4007204F5177156
:1015B00004F13800FFF72EFF03B030BDAC3B00084C
:1015C00010B52023044683F31188FFF7A9FD0223F9
:1015D0002374002383F3118810BD000038B5C3695C
:1015E00004460D461BB904210844FFF793FF294622
:1015F00004F11400FFF79AFE002806DA201D4FF4CC
:101600008061BDE83840FFF785BF38BD0268436898
:101610001143016003B118477047000013B5446BD4
:10162000D4F894341A681178042915D1217C022940
:1016300012D11979128901238B4013420CD101A9CF
:1016400004F14C0001F054FED4F89444019B21793C
:101650000246206800F0DAF902B010BD143001F043
:10166000D7BD00004FF0FF33143001F0D1BD0000B2
:101670004C3001F0A9BE00004FF0FF334C3001F0B8
:10168000A3BE0000143001F0A5BD00004FF0FF31F3
:10169000143001F09FBD00004C3001F075BE000019
:1016A0004FF0FF324C3001F06FBE0000D0F89424B0
:1016B00038B5136819780429054601D0012038BDD2
:1016C000017C0229FAD112795C8901209040044002
:1016D000F4D105F1140001F037FD02460028EDD0E9
:1016E000D5F894544FF480732868697900F07CF938
:1016F000204638BD406BFFF7D9BF0000002070477F
:10170000704700007FB5124B036000234360836085
:10171000C360012502260F4B057404460290019315
:1017200000F18402294600964FF48073143001F0D2
:10173000E7FC094B0193029400964FF4807304F583
:101740002372294604F14C0001F0AEFD04B070BDD7
:10175000D43B0008F51600081D1600080B6820226F
:1017600082F311880A7903EB820290614A79093287
:1017700043F822008A7912B103EB820398610223B5
:101780000374C0F89414002383F311887047000099
:1017900038B5037F044613B190F85430ABB9201D1F
:1017A00001250221FFF732FF04F1140025776FF0C5
:1017B000010100F087FC84F8545004F14C006FF0F4
:1017C0000101BDE8384000F07DBC38BD10B50121F5
:1017D00004460430FFF71AFF0023237784F85430BF
:1017E00010BD000038B504460025143001F0A0FCFF
:1017F00004F14C00257701F06FFD201D84F8545052
:101800000121FFF703FF2046BDE83840FFF74EBF38
:1018100090F8443003F06003202B19D190F8452054
:10182000212A0AD0222A4FF000030ED0202A0FD1FD
:10183000084A82630722C26304E0064B83630723DE
:10184000C36300230364012070478363C363F9E724
:101850000020704701240020D0F8943437B51A686E
:101860001178042904461AD1017C022917D119796B
:10187000128901238B40134211D100F14C052846F7
:1018800001F0EAFD58B101A9284601F031FDD4F874
:101890009444019B21790246206800F0B7F803B018
:1018A00030BD000000EB8103F7B59C6905460E468C
:1018B000F4B1202383F3118805EB8607201D08214E
:1018C000FFF7A4FEFB685B691B684C3413B120462C
:1018D00001F01CFD01A9204601F00AFD024648B1B5
:1018E000019B3146284600F091F8002383F31188CC
:1018F00003B0F0BDFB685A691268002AF5D01B8A54
:10190000013B1340F1D105F14402EAE7093138B552
:1019100050F82140DCB1202383F31188D4F89424BB
:101920001368527903EB8203DB689B695D6845B1FC
:1019300004216018FFF76AFE294604F1140001F043
:101940000DFC2046FFF7B2FE002383F3118838BD5B
:101950007047000000F0CEBF0123037000234360F6
:10196000C36183620362C362436203630381438191
:101970007047000038B50446202383F31188002502
:101980004160C56005614561856100F0C3FF0223C8
:10199000237085F3118838BD70B500EB81030546CF
:1019A0005069DA600E46144618B110220021FFF784
:1019B00059FAA06918B110220021FFF753FA3146F5
:1019C0002846BDE8704001F06FB80000028902F0BF
:1019D00001020281428902F0010242810022026179
:1019E0004261826101F0F4B8F0B400EB81044789F0
:1019F000E4680125A4698D403D43458123600023AF
:101A0000A2606360F0BC01F00FB90000F0B400EB1D
:101A100081040789E468012564698D403D4305819F
:101A200023600023A2606360F0BC01F089B900006C
:101A300070B50223002504460370A0F84C5080F8CE
:101A40004E5080F84F5005814581C5600561456164
:101A5000856180F8345000F0C3FF63681B6823B1D0
:101A600029462046BDE87040184770BD436802789B
:101A70001B6880F85020052202700BB10421184722
:101A800070470000436890F850201B6802700BB14B
:101A9000052118477047000090F8343070B50446AF
:101AA00013B1002380F8343004F14402204601F0E1
:101AB000B1F863689B6863BB94F8445015F0600606
:101AC00015D194F8453005F07F0545EA032540F22D
:101AD00002339D4200F00E815BD8022D00F0DC80C5
:101AE0003FD8002D00F08780012D00F0CF8000212D
:101AF000204601F0E7FA0021204601F0D9FA636898
:101B00001B6813B1062120469847062384F8343019
:101B100070BD204698470028CED094F84B2094F80A
:101B20004A3043EA0223E26B934238BFE36394F9FD
:101B30004430E56B002B4FF0200380F2FD80002D38
:101B400000F0EC80092284F8342083F3118800210E
:101B5000E36BA26B2046FFF759FF002383F3118844
:101B600070BDB5F5817F00F0B180B5F5407F49D0FB
:101B7000B5F5807FBBD194F84630012BB7D1B4F8CE
:101B80004C3023F00203A4F84C30A663E6632664CD
:101B9000C3E740F201639D421ED8B5F5C06F3BD24A
:101BA000B5F5A06FA3D1B4F84430B3F5A06F0ED152
:101BB00094F8463084F84E30204600F069FF6368A0
:101BC0001B6813B10121204698470323237000238B
:101BD000A363E3632364A0E7B5F5106F32D040F64A
:101BE00002439D4252D0B5F5006F80D104F14F03FE
:101BF000A363012324E004F14C03A3630223E36302
:101C000025648AE794F84630012B7FF470AFB4F86E
:101C10004C3043F00203B6E794F84920616894F829
:101C200048304D6894F8471043EA0223204694F860
:101C30004620A84700283FF45AAF4368A3630368CF
:101C4000E363A4E72378042B10D1202383F31188C6
:101C50002046FFF7BBFE86F31188636884F84F6067
:101C60001B68032121700BB12046984794F8463039
:101C7000002BACD084F84F300423237063681B68BA
:101C8000002BA4D0022120469847A0E7374BA3633E
:101C90000223E36300239DE794F8481011F0800FBE
:101CA000204601F00F010ED000F0A6FF012806D05B
:101CB00002287FF41CAF2E4BA363E06367E72D4B34
:101CC000A363E56363E700F089FFEFE794F846302C
:101CD000002B7FF40CAF94F8483013F00F013FF461
:101CE00076AF1A06204602D501F000FA6FE701F040
:101CF000F3F96CE794F84630002B7FF4F8AE94F8D3
:101D0000483013F00F013FF462AF1B06204602D5A6
:101D100001F0D8F95BE701F0CBF958E7142284F819
:101D2000342083F311882B462A4629462046FFF7A4
:101D30005BFE85F3118870BD5DB1152284F83420F7
:101D400083F311880021E36BA26B2046FFF74CFE62
:101D500003E70B2284F8342083F311882B462A46AC
:101D600029462046FFF752FEE3E700BF043C000887
:101D7000FC3B0008003C000838B590F834300446BD
:101D8000152B29D8DFE803F03E28282828283E28EC
:101D9000280B293928282828282828283E3E90F86A
:101DA0004B1090F84A20C36B42EA01229A4214D9A0
:101DB000C268128AB3FBF2F502FB15356DB9202318
:101DC00083F311882B462A462946FFF71FFE85F329
:101DD00011880A2384F8343038BD142384F8343051
:101DE000202383F3118800231A4619462046FFF763
:101DF000FBFD002383F3118838BD036C03B19847C2
:101E00000023E7E7002101F05DF90021204601F001
:101E10004FF963681B6813B10621204698470623D3
:101E2000D8E7000090F83420152A38B5044622D8A7
:101E30000123934040F6416213421DD113F48015F3
:101E40000FD19B0217D50B2380F83430202383F366
:101E500011882B462A462946FFF7D8FD85F31188BD
:101E600038BDC3689B695B682BB9036C03B19847A5
:101E7000002384F8343038BD002101F023F900211B
:101E8000204601F015F963681B6813B1062120464E
:101E900098470623EDE70000024B00221B605B60C1
:101EA0009A607047D4360020002303748268054B83
:101EB0001B6899689142FBD25A68036042601060C7
:101EC00058607047D436002008B5202383F311886A
:101ED000037C032B05D0042B0DD02BB983F3118881
:101EE00008BD436900221A604FF0FF334361FFF7DA
:101EF000DBFF0023F2E790E80C001A6002685360F1
:101F0000F2E70000002303748268054B1B689968A0
:101F10009142FBD85A680360426010605860704775
:101F2000D4360020054B19690874186802681A60D5
:101F30005360186101230374FEF7E6B9D43600201C
:101F400030B54B1C87B005460A4C10D023690A4AAD
:101F500001A800F0D3F82846FFF7E4FF049B13B173
:101F600001A800F007F92369586907B030BDFFF7F1
:101F7000D9FFF8E7D4360020C91E000838B50C4D4B
:101F800041612B6981689A689142044603D8BDE893
:101F90003840FFF789BF1846FFF786FF01232C6101
:101FA000014623742046BDE83840FEF7ADB900BFB6
:101FB000D4360020044B1A681B6990689B689842CD
:101FC00094BF002001207047D436002010B5084C83
:101FD000236820691A6822605460012223611A7400
:101FE000FFF790FF01462069BDE81040FEF78CB96D
:101FF000D4360020826002220274002242747047AC
:102000008368A3F17C0243F80C2C026943F83C2C52
:10201000426943F8382C074A43F81C2CC26843F83D
:10202000102C022203F8082C002203F8072CA3F13D
:10203000180070472103000810B5202383F311888E
:10204000FFF7DEFF00210446FFF798FF002383F32C
:102050001188204610BD0000024B1B6958610F20FB
:10206000FFF760BFD4360020202383F31188FFF7E9
:10207000F3BF000008B50146202383F31188082030
:10208000FFF75EFF002383F3118808BD49B1064BBB
:1020900042681B6918605A60136043600420FFF7B0
:1020A0004FBF4FF0FF307047D4360020036898428E
:1020B00006D01A680260506059611846FFF7F4BEF6
:1020C0007047000038B504460D462068844200D1B0
:1020D00038BD036823605C604561FFF7E5FEF4E707
:1020E000054B03F114025A619A614FF0FF32DA6135
:1020F00000221A62704700BFD4360020F8B5036191
:102100001A4BC2605C6A1A4B1A46022952F8145FD5
:1021100038BF0221954206461F460AD15861986190
:102120001C620560456081600819BDE8F84001F057
:10213000B5B9186AAB68241A0C1902D3E41A2D68D1
:1021400004E09C4202D2204401F0B8F9AB689C4202
:10215000F4D86B68736035601E606E60B460A96807
:102160004FF0FF33091BA960FB61F8BD000C004074
:10217000D436002010B41A4C234653F8141F814261
:1021800010D0416802680A60026851609A424FF0BC
:102190000001C16003D0936881680B4493605DF8CF
:1021A000044B70470A68626100209A425360C8601D
:1021B00003D15DF8044B01F07BB993688868034450
:1021C0009360084A206A526A121A9342E7D9991A10
:1021D000012998BF931C18445DF8044B01F06EB9B7
:1021E000D4360020000C004000207047FEE70000BD
:1021F000704700004FF0FF3070470000022906D002
:10220000032906D00129064818BF00207047054859
:102210007047032A9ABF044800EBC20000207047B1
:10222000D83C00088C3C00080824002070B59AB007
:1022300001AD064608462946144600F095F82846A2
:10224000FEF708FEC0B2431C5B0086E8180023704E
:1022500003236370002302341946DAB2904204F17A
:10226000020401D81AB070BDEA5C04F8022C04F82C
:10227000011C0133F1E7000008B5202383F3118826
:102280000348FFF7E9FA002383F3118808BD00BF74
:102290001437002010B50446052916D8DFE801F0F0
:1022A00016150316161D202383F311880E4A0121EB
:1022B000FFF772FB20460D4A0221FFF76DFB0C4829
:1022C000FFF790FA002383F3118810BD202383F3D6
:1022D00011880748FFF75CFAF4E7202383F311889D
:1022E0000348FFF773FAEDE7083C00082C3C0008B0
:1022F0001437002038B50C4D0C4C0D492A4604F11A
:102300000800FFF793FF05F1CA0204F11000094924
:10231000FFF78CFF05F5CA7204F118000649BDE805
:102320003840FFF783BF00BFDC3B002008240020BB
:10233000583C0008653C0008733C000870B5044632
:1023400008460D46FEF786FDC6B2204601340378E6
:102350000BB9184670BD32462946FEF763FD0028CA
:10236000F3D1012070BD00002DE9F84F05460C4661
:10237000FEF770FD2B49C6B22846FFF7DFFF08B114
:102380000336F6B228492846FFF7D8FF08B11036C1
:10239000F6B2632E0DD8DFF88C80DFF88C90234FD7
:1023A000DFF890A0DFF890B02E7846B92670BDE82F
:1023B000F88F29462046BDE8F84F01F0A1BB252E35
:1023C0002CD1072241462846FEF72CFD58B9DBF8F0
:1023D00000302360DBF804306360BBF808302381F1
:1023E00007350A34E0E7082249462846FEF71AFD79
:1023F000A0B90F4BA21C13F8011F09095345C95D71
:1024000002F8021C197801F00F0102F10202C95D05
:1024100002F8031CEFD118340835C5E726700135E2
:102420000134C1E7F83C0008733C00080B3D00088C
:102430000F7AFF1F1B7AFF1F003D0008BFF34F8F6D
:10244000024AD368DB03FCD4704700BF003C024063
:1024500008B5094B1B7873B9FFF7F0FF074B1A69F2
:10246000002ABFBF064A5A6002F188325A601A68D1
:1024700022F480621A6008BD3A3E0020003C02400F
:102480002301674508B50B4B1B7893B9FFF7D6FFBF
:10249000094B1A6942F000421A611A6842F48052EC
:1024A0001A601A6822F480521A601A6842F4806234
:1024B0001A6008BD3A3E0020003C0240172870B563
:1024C00013D80B4A0B4C137863B90B4E4FF00061D5
:1024D00044F8231056F823500133182B2944F7D120
:1024E0000123137054F8200070BD002070BD00BFA0
:1024F0009C3E00203C3E00201C3D0008014B53F850
:10250000200070471C3D000818207047172810B5A0
:10251000044601D9002010BDFFF7D0FF064B53F849
:1025200024301844C21A0BB9012010BD12680132C0
:10253000F0D1043BF6E700BF1C3D0008172810B59A
:10254000044629D8FFF77AFFFFF782FF1349F323E8
:10255000CB600C23B0FBF3F203FB1200D30143EA80
:10256000C003DBB243F4007343F002030B610B6959
:1025700043F480330B61FFF761FF2046FFF79EFFB6
:10258000074B53F8241000F0D9F8FFF77BFF2046E3
:10259000BDE81040FFF7BABF002010BD003C02406C
:1025A0001C3D00082DE9F84312F00103154640D107
:1025B0008218B2F1026F3CD22C4B1B6813F001035E
:1025C00037D02B4CFFF744FFF323E360FFF736FFD0
:1025D00040F20127032D01D9830713D0244C0F4665
:1025E000401A40F20118EB1B0B44012B00EB0706CD
:1025F000236924D823F001032361FFF743FF01205F
:10260000BDE8F883236923F44073236123693B43C6
:10261000236151F8046B0660BFF34F8FFFF70EFF85
:1026200003689E4208D0236923F001032361FFF76A
:1026300029FF0020BDE8F883043D0430CAE723F4F5
:1026400040732361236943EA08032361B94637F8DD
:10265000023B3380BFF34F8FFFF7F0FE3688B9F8A7
:102660000030B6B2B342BED0DDE700BF0038024052
:10267000003C0240084908B50B7828B153B9FFF770
:10268000E7FE01230B7008BD23B1BDE808400870C8
:10269000FFF7F8BE08BD00BF3A3E002010B5024467
:1026A000064B0439D2B2904200D110BD441C00B296
:1026B00053F8200041F8040FE0B2F4E7502800403E
:1026C000104B30B51C6F240407D41C6F44F4007405
:1026D0001C671C6F44F400441C670B4C236843F4D4
:1026E000807323600244094B0439D2B2904200D176
:1026F00030BD441C00B251F8045F43F82050E0B2F2
:10270000F4E700BF0038024000700040502800404D
:1027100007B5012201A90020FFF7C0FF019803B00F
:102720005DF804FB07B502A9012241F8040D002061
:10273000FFF7C6FF03B05DF804FB00007047000020
:10274000034B1B689B0042BF024B01221A7070476B
:10275000743802409D3E0020014B1878704700BF3E
:102760009D3E0020064A536823F001035360EFF3B7
:102770000983683383F30988002383F31188704742
:1027800030EF00E010B5202383F31188104B5B6815
:1027900013F4006318D0F1EE103AEFF309844FF010
:1027A000807344F84C3C0B4BDB6844F8083CA4F1C4
:1027B000680383F30988FFF7FDFB18B1064B44F863
:1027C000503C10BD054BFAE783F3118810BD00BFE4
:1027D00000ED00E030EF00E03103000834030008B2
:1027E00070470000FEE70000084A094B09498B4288
:1027F00004D3094A0021934205D3704752F8040FCD
:1028000043F8040BF3E743F8041BF4E7F43E000835
:10281000904100209041002090410020836D30B510
:1028200000229D68446D11464FF0FF3004EB4213C7
:1028300001329542C3F80019C3F81019C3F808090A
:10284000C3F8001BC3F8101BC3F8080BEED24FF0FF
:102850000113C4F81C3830BD890141F02001016129
:1028600003699B06FCD4122000F0B4BE204B03EB9E
:1028700080022DE9F047D2F80CE05D6DDEF81420FF
:10288000461CD2F800C005EB063605EB401851682F
:1028900061450BD3D5F83428012303FA00F022EA6E
:1028A0000000C5F834081846BDE8F087BEF81040AF
:1028B000ACEB0103A34228BF2346D8F81849A4B2C1
:1028C000B3EB840F10D894681F46A4F1040959F89B
:1028D00004AFC6F800A0042F01D9043FF7E71C4459
:1028E0000B4494605360D2E70020BDE8F08700BF3E
:1028F000A03E002010B5054C2046FFF72DF84FF004
:10290000A0436365024BA36510BD00BFA03E00203D
:10291000A03D00080378012B70B5054650D12A4B25
:10292000446D98421BD1294B5A6B42F080025A6386
:102930005A6D42F080025A655A6D5A6942F080021F
:102940005A615A6922F080025A610E2143205B6964
:10295000FEF76CFC1E4BE3601E4BC4F800380023EE
:10296000C4F8003EC02323606E6D4FF45023A36370
:102970003369002BFCDA012333610C2000F02AFEBE
:102980003369DB07FCD4122000F024FE3369002BEE
:10299000FCDA0026A6602846FFF740FF6B68C4F803
:1029A0001068DB68C4F81468C4F81C684BB90A4B9B
:1029B000A3614FF0FF336361A36843F00103A36099
:1029C00070BD064BF4E700BFA03E00200038024077
:1029D0004014004003002002003C30C0083C30C0DE
:1029E000F8B5446D054600212046FFF735FFA96D77
:1029F00000234FF001128F68C4F834384FF000669E
:102A0000C4F81C284FF0FF3004EB431201339F42FF
:102A1000C2F80069C2F8006BC2F80809C2F8080BD6
:102A2000F2D20B686A6DEB6563621023136116695D
:102A300016F01006FBD1122000F0CCFDD4F80038BF
:102A400023F4FE63C4F80038A36943F4402343F041
:102A50001003A3610923C4F81038C4F814380A4BD2
:102A6000EB604FF0C043C4F8103B084BC4F8003B88
:102A7000C4F81069C4F80039EB6D03F1100243F497
:102A80008013EA65A362F8BD7C3D00084080001019
:102A9000426D90F84E10D2F8003823F4FE6343EAFA
:102AA0000113C2F8003870472DE9F0410EB200EB77
:102AB00086080D46D8F80C100F6807F00303022BA8
:102AC00050D0032B50D03D4A3D4F012B18BF174625
:102AD000446D4FEA451E04EB0E030022C3F8102B91
:102AE0008A6905F1100C002A40D04A8A05F1580382
:102AF0005B013A43E2500123D4F81C2803FA0CF39B
:102B00001343A6444A69C4F81C380023CEF8103990
:102B100005F13F03002A39D00A8A898B92080129DE
:102B200088BF4A43C16D04EB8303561841EA024251
:102B3000C66529465A602046FFF78EFED8F80C304D
:102B40001B8A43EA85531F4305F148035B01E750A5
:102B50000123D4F81C2803FA05F51543C4F81C58C2
:102B6000BDE8F081174FB3E7174FB1E704EB461309
:102B7000D3F8002B22F40042C3F8002BD4F81C2811
:102B8000012303FA0CF322EA0303BAE704EB8303FD
:102B90000E4A5A6004EB461629462046FFF75CFEB3
:102BA000D6F8003923F40043C6F80039D4F81C38AD
:102BB000012202FA05F523EA0505CFE7008000109F
:102BC000008004100080081000800C100004000237
:102BD000826D1268C265FFF721BE00005831436D57
:102BE00049015B5813F4004004D013F4001F14BFD4
:102BF00001200220704700004831436D49015B58B5
:102C000013F4004004D013F4001F14BF012002206D
:102C10007047000000EB8101CB68196A0B681360F4
:102C20004B6853607047000000EB810330B5DD68EE
:102C3000AA691368D36019B9402B84BF402313607D
:102C40006B8A1468426D1C44013CB4FBF3F463438B
:102C5000033323F0030302EB411043EAC44343F080
:102C6000C043C0F8103B2B6803F00303012B09B2EB
:102C70000ED1D2F8083802EB411013F4807FD0F85F
:102C8000003B14BF43F0805343F00053C0F8003BB7
:102C900002EB4112D2F8003B43F00443C2F8003B80
:102CA00030BD00002DE9F041244D6E6D06EB401360
:102CB0000446D3F8087BC3F8087B38070AD5D6F852
:102CC0001438190706D505EB84032146DB6828462E
:102CD0005B689847FA072FD5D6F81438DB072BD551
:102CE00005EB8403D968CCB98B69488A5E68B6FB6A
:102CF000F0F200FB12628AB91868DA6890420DD2CD
:102D0000121A83E81400202383F311880B4821460C
:102D1000FFF78AFF84F31188BDE8F081012303FAED
:102D200004F26B8923EA02036B81CB6823B121464D
:102D30000248BDE8F0411847BDE8F081A03E002000
:102D400000EB810370B5DD68436D6C692668E66051
:102D50004A0156BB1A444FF40020C2F810092A68F1
:102D600002F00302012A0AB20ED1D3F8080803EBDD
:102D7000421410F4807FD4F8000914BF40F0805052
:102D800040F00050C4F8000903EB4212D2F80009E9
:102D900040F00440C2F80009D3F83408012202FAD6
:102DA00001F10143C3F8341870BD19B9402E84BF36
:102DB0004020206020682E8A841940F00050013C99
:102DC0001A44B4FBF6F440EAC440C6E7F8B504463A
:102DD0001E48456D05EB4413D3F80869C3F808692C
:102DE000F10717D5D5F81038DA0713D500EB8403AF
:102DF000D9684B691F68DA68974218D2D21B00273E
:102E00001A605F60202383F311882146FFF798FF43
:102E100087F31188330617D5D5F834280123A3404A
:102E2000134211D02046BDE8F840FFF71FBD012333
:102E300003FA04F2038923EA020303818B68002B5F
:102E4000E8D021469847E5E7F8BD00BFA03E002046
:102E500096482DE9F84F456D6E69AB691E4016F432
:102E6000805F6E61044605D0FEF7E2FDBDE8F84FD5
:102E7000FFF788BC002E12DAD5F8003E8B489B077E
:102E80001EBFD5F8003E23F00303C5F8003ED5F879
:102E9000043823F00103C5F80438FEF7F3FD3705C5
:102EA00002D58248FEF7E2FDB0040CD5D5F808380B
:102EB00013F0060FEB6823F470530CBF43F4105368
:102EC00043F4A053EB60310704D56368DB680BB1B2
:102ED00076489847F2025AD4B3020CD5D4F85480FD
:102EE000DFF8C8A100274FF00109A36D9B68F9B274
:102EF0008B4280F08780F70619D5616D0A6AC2F3AC
:102F00000A1702F00F0302F4F012B2F5802F00F05E
:102F1000A180B2F5402F0AD104EB830301F5805163
:102F2000DB68186A00231A469F4240F0878030030E
:102F3000D5F8184813D5E10302D50020FFF7B2FEFB
:102F4000A20302D50120FFF7ADFE630302D50220E4
:102F5000FFF7A8FE270302D50320FFF7A3FE7503A2
:102F600084D5E00702D50020FFF730FFA10702D586
:102F70000120FFF72BFF620702D50220FFF726FF93
:102F800023077FF573AF0320FFF720FF6EE7D4F828
:102F90005480DFF818A100274FF00109A36D9B684A
:102FA0005FFA87FB5B4597D308EB4B13D3F80029F7
:102FB00002F44022B2F5802F22D1D3F80029002A52
:102FC0001EDAD3F8002942F09042C3F80029D3F862
:102FD0000029002AFBDB5946606DFFF73DFC228982
:102FE00009FA0BF322EA0303238104EB8B03DB686A
:102FF0009B6813B15946504698475846FFF736FC30
:103000000137CBE708EB4112D2F8003B03F4402331
:10301000B3F5802F10D1D2F8003B002B0CDA628977
:1030200009FA01F322EA0303638104EB8103DB68FD
:10303000DB680BB150469847013756E79C0708BF3D
:103040000A68072B98BF027003F101039CBF120AA4
:10305000013069E7023304EB830201F580515268C5
:1030600090690268D0F808C04068A2EB000E002208
:10307000104697420AD104EB830463689B699A68FF
:103080003A449A605A6817445F6050E712F0030FA1
:1030900008BF0868964588BF8CF8000002F101025D
:1030A00084BF000A0CF1010CE3E700BFA03E002042
:1030B000436D03EB4111D1F8003B43F40013C1F819
:1030C000003B7047436D03EB4111D1F8003943F4E5
:1030D0000013C1F800397047436D03EB4111D1F87B
:1030E000003B23F40013C1F8003B7047436D03EB32
:1030F0004111D1F8003923F40013C1F800397047A9
:1031000030B5039C0172043304FB0325C361049BA7
:1031100003630021059B00604060C1604261026161
:103120008561046242628162C162436330BD000016
:103130000022416A41610161C2608262C2626FF035
:103140000101FEF7BFBF000003694269934203D14A
:10315000C2680AB100207047181D704703691960E2
:10316000C2680132C260C26913448269036193423A
:1031700024BF436A03610021FEF798BF38B50446B7
:103180000D46E3683BB16269131D1268A3621344E4
:10319000E362002038BD237A33B929462046FEF782
:1031A00075FF0028EDDA38BD6FF00100FBE7000085
:1031B000C368C269013BC3604369134482694361C8
:1031C000934224BF436A436100238362036B03B1CC
:1031D0001847704770B52023044683F31188866A28
:1031E0003EB9FFF7CBFF054618B186F31188284694
:1031F00070BDA36AE26A13F8015BA362934202D333
:103200002046FFF7D5FF002383F31188EFE7000086
:103210002DE9F84F04460E4690469946202787F33D
:1032200011880025AA46D4F828B0BBF1000F09D1B7
:1032300049462046FFF7A2FF20B18BF311882846AC
:10324000BDE8F88FA16AE36AA8EB050B5B1A9B4502
:1032500028BF9B46BBF1400F1BD9334601F140020A
:1032600051F8040B43F8040B9142F9D1A36A40339F
:103270004036A3624035A26AE36A9A4202D32046EE
:10328000FFF796FF8AF311884545D8D287F3118856
:10329000C9E730465A46FDF7BBFDA36A5B445E446E
:1032A000A3625D44E7E7000010B5029C017204339D
:1032B00003FB0421C36100238362C362039B036396
:1032C000049B00604060C4604261026181610462ED
:1032D0004262436310BD0000026AC260426A4261FA
:1032E000026100228262C2626FF00101FEF7EABE53
:1032F000436902699A4203D1C2680AB1002070474B
:10330000184650F8043B0B6070470000C368C26960
:103310000133C3604369134482694361934224BF0C
:10332000436A43610021FEF7C1BE000038B5044680
:103330000D46E3683BB123691A1DA262E26913449A
:10334000E362002038BD237A33B929462046FEF7D0
:103350009DFE0028EDDA38BD6FF00100FBE70000AC
:1033600003691960C268013AC260C2691344826984
:103370000361934224BF436A036100238362036BAA
:1033800003B118477047000070B5202304460E466D
:1033900083F31188856A35B91146FFF7C7FF10B16D
:1033A00085F3118870BDA36A1E70A36AE26A0133B7
:1033B0009342A36204D3E16920460439FFF7D0FFAA
:1033C000002080F3118870BD2DE9F84F04460D46AA
:1033D00091469A464FF0200888F311880026B3469C
:1033E000A76A4FB951462046FFF7A0FF20B187F3E7
:1033F00011883046BDE8F88FA06AE76AA9EB06039A
:103400003F1A9F4228BF1F46402F1BD905F140039A
:1034100055F8042B40F8042B9D42F9D1A36A4033A0
:10342000A3624036A26AE36A9A4204D3E169204665
:103430000439FFF795FF8BF311884E45D9D288F3F5
:103440001188CDE729463A46FDF7E2FCA36A3B44E2
:103450003D44A3623E44E5E7026943699A4203D1D1
:10346000C3681BB9184670470023FBE7836A002B2B
:10347000F8D0043B9B1AF5D01360C368013BC360CE
:10348000C3691A44836902619A4224BF436A036193
:10349000002383620123E5E700F034B9034B0022E7
:1034A00058631A610222DA60704700BF000C0040C6
:1034B000014B0022DA607047000C0040014B58635A
:1034C000704700BF000C0040FEE7000010B5174C2D
:1034D000FEF7E2FCFEF704FE802215492046FEF7C7
:1034E00089FD012344F8180C0374124B124AD96861
:1034F00021F4E0610904090C0A431049DA60CA6842
:1035000042F08072CA600E490A6842F001020A6005
:103510001022DA77202283F82220002383F31188F7
:1035200062B60848BDE81040FEF786BDFC360020B4
:10353000AC3D000800ED00E00003FA05F0ED00E00E
:10354000001000E0B43D00082DE9F84F1F4CDFF8F3
:103550008090656904F114074FF00008D9F8243011
:10356000266AAA689E1B96421DD34FF0200AAA68BD
:10357000236AD5F80CB0134423622B68BB425F600A
:10358000A6EB02066361C5F80C8001D1FFF790FF3E
:1035900088F311882869D8478AF311886569AB6870
:1035A0009E42E4D2DAE76269BA420CD091682362A3
:1035B0008E1B9660A86802282CBF1818981CBDE8BE
:1035C000F84FFFF77BBFBDE8F88F00BFD43600206F
:1035D000000C0040034B59685A68521A9042FBD8BD
:1035E000704700BF001000E04B6843608B68836049
:1035F000CB68C3600B6943614B6903628B694362AB
:103600000B6803607047000008B5224B22481A6916
:1036100040F2FF110A431A611A6922F4FF7222F084
:1036200001021A611A691A6B0A431A631A6D0A4376
:103630001A651A4A1B6D1146FFF7D6FF184802F1AA
:103640001C01FFF7D1FF174802F13801FFF7CCFF4B
:10365000154802F15401FFF7C7FF144802F1700149
:10366000FFF7C2FF124802F18C01FFF7BDFF1148BE
:1036700002F1A801FFF7B8FF0F4802F1C401FFF7FC
:10368000B3FF0E4802F1E001FFF7AEFFBDE80840CE
:1036900000F0A4B80038024000000240D43D000809
:1036A0000004024000080240000C024000100240EA
:1036B0000014024000180240001C0240002002409A
:1036C00008B500F0FFF9FFF701FFFFF739F8BDE893
:1036D0000840FEF70FBE000070470000084B1A6953
:1036E000920710B508D500241C61202383F31188AC
:1036F000FFF72AFF84F31188BDE81040FFF742B8B6
:10370000000C0040104B1A6C42F008021A641A6E4A
:1037100042F008021A660D4A1B6E936843F00803D4
:1037200093600B4B53229A624FF0FF32DA62002211
:103730009A615A63DA605A6001225A6108211A605C
:103740003220FDF773BD00BF00380240002004E0C6
:10375000000C00401F4B1A696FEAC2526FEAD25246
:103760001A611A69C2F308021A614FF0FF301A6930
:103770005A69586100215A6959615A691A6A62F096
:1037800080521A621A6A02F080521A621A6A5A6ADF
:1037900058625A6A59625A6A1A6C42F080521A6424
:1037A0001A6E42F080521A661A6E0B4A106840F484
:1037B00080701060186F00F44070B0F5007F1EBF7D
:1037C0004FF4803018671967536823F4007353600F
:1037D00000F058B90038024000700040324B4FF002
:1037E00080521A64314A4FF4404111601A6842F025
:1037F00001021A601A689207FCD59A6822F0030247
:103800009A60294B19469A6812F00C02FBD118688D
:1038100000F0F90018609A601A6842F480321A6069
:103820000B689B03FCD54B6F43F001034B671E4BAA
:103830005A6F9007FCD51E4A5A601A6842F080728F
:103840001A601A4A53685904FCD5174B1A6892013A
:10385000FCD5184A9A600322C3F88C20164B1A68CC
:10386000164B9A42164B1BD1164A1168164A9142C2
:1038700016D140F205121A600B4B9A6842F0020210
:103880009A609A6802F00C02082AFAD15A6C42F443
:1038900080425A645A6E42F480425A665B6E7047A8
:1038A00040F20572E7E700BF0038024000700040B8
:1038B0001854400700948838002004E01164002068
:1038C000003C024000ED00E041C20F41084A08B54B
:1038D000536911680B4003F00103536123B1054A9A
:1038E00013680BB150689847BDE80840FEF74ABF1F
:1038F000003C014010410020084A08B55369116896
:103900000B4003F00203536123B1054A93680BB1E6
:10391000D0689847BDE80840FEF734BF003C01403E
:1039200010410020084A08B5536911680B4003F0A4
:103930000403536123B1054A13690BB150699847D9
:10394000BDE80840FEF71EBF003C014010410020CA
:10395000084A08B5536911680B4003F00803536126
:1039600023B1054A93690BB1D0699847BDE8084077
:10397000FEF708BF003C014010410020084A08B58E
:10398000536911680B4003F01003536123B1054ADA
:10399000136A0BB1506A9847BDE80840FEF7F2BEC3
:1039A000003C014010410020174B10B55C691A68BB
:1039B000144004F478725A61A30604D5134A936A3A
:1039C0000BB1D06A9847600604D5104A136B0BB14F
:1039D000506B9847210604D50C4A936B0BB1D06B02
:1039E0009847E20504D5094A136C0BB1506C98470F
:1039F000A30504D5054A936C0BB1D06C9847BDE87C
:103A00001040FEF7BFBE00BF003C01401041002047
:103A10001A4B10B55C691A68144004F47C425A6170
:103A2000620504D5164A136D0BB1506D98472305F6
:103A300004D5134A936D0BB1D06D9847E00404D5BB
:103A40000F4A136E0BB1506E9847A10404D50C4A6F
:103A5000936E0BB1D06E9847620404D5084A136F79
:103A60000BB1506F9847230404D5054A936F0BB1EF
:103A7000D06F9847BDE81040FEF784BE003C01407F
:103A800010410020062108B50846FDF7CFFB0621AE
:103A90000720FDF7CBFB06210820FDF7C7FB062119
:103AA0000920FDF7C3FB06210A20FDF7BFFB062115
:103AB0001720FDF7BBFB06212820BDE80840FDF7D5
:103AC000B5BB000008B5FFF745FE00F00DF8FDF7A7
:103AD00053FDFDF73FFFFDF713FEFFF7FDFDBDE8CA
:103AE0000840FFF7D9BC0000002304491A465A5089
:103AF000C8180833802B4260F9D17047104100206C
:103B0000034611F8012B03F8012B002AF9D1704765
:103B1000121012131211000053544D3332463F3F1E
:103B20003F000000012033000010410101105A0144
:103B3000031059010710310100000000183B000874
:103B40003F00000013040000783B00083F00000025
:103B500019040000823B00083F000000210400001F
:103B60008C3B00083F000000143700209C290020F7
:103B7000042E00206C32002053544D333246343032
:103B8000780053544D3332463432780053544D3319
:103B900032463434365858000096000000000000C9
:103BA0000000000000000000000000000000000015
:103BB000411500082D150008691500085515000865
:103BC000611500084D150008391500082515000875
:103BD0007515000800000000791600086516000839
:103BE000A11600088D160008991600088516000811
:103BF000711600085D160008FD16000800000000A0
:103C000001000000000000000200000000000000B1
:103C1000A51800080D19000840004000AC3B00202A
:103C2000BC3B002002000000000000000300000078
:103C30000000000051190008000000001000000002
:103C4000CC3B00200000000001000000000000004C
:103C5000A03E0020010102004865782F50726F6677
:103C600069434E430043756265426C61636B2B2D63
:103C7000424C002553455249414C250095220008ED
:103C8000FD210008111800087922000843000000F7
:103C9000943C000809024300020100C032090400FC
:103CA00000010202010005240010010524010001A9
:103CB000042402020524060001070582030800FF10
:103CC00009040100020A000000070501024000008B
:103CD000070581024000000012000000E03C0008DF
:103CE0001201100102000040AE2D0111000201027C
:103CF000030100000403090425424F4152442500FA
:103D000043756265426C61636B2B00303132333432
:103D100035363738394142434445460000400000BB
:103D200000400000004000000040000000000100D2
:103D3000000002000000020000000200000002007B
:103D4000000002000000020000000200004000002D
:103D500000400000004000000040000000000100A2
:103D6000000002000000020000000200000002004B
:103D7000000002000000020000000200000000003D
:103D8000991A0008791D0008251E0008400040000F
:103D9000003F0020003F002001000000103F0020F5
:103DA0008000000040010000030000006D61696EAA
:103DB00000000000CC3D0008183F0020104100200A
:103DC00001000000C93400080000000069646C654F
:103DD000000000000000812A00020000AAAAAAAA8E
:103DE00000000000FFFF00000000000000A00A002B
:103DF0000000000000000000AAAAAAAA000000001B
:103E0000FFFF0000000000000000000000000000B4
:103E100000000000AAAAAAAA00000000FFFF0000FC
:103E2000000000000000000080298A01000000005E
:103E3000AAAAAAAA40154501FFFF0000007070075A
:103E4000777000004080020100000000AAAAAAAA20
:103E500000400100F7FF00000000008008000000A3
:103E60000000000000000000AAAAAAAA00000000AA
:103E7000FFFF000000000000000000000000000044
:103E800000000000AAAAAAAA00000000FFFF00008C
:103E90000000000000000000000000000000000022
:103EA0000A00000000000000030000000000000005
:103EB0000000000000000000000000000000000002
:103EC00000000000000000000000000000000000F2
:103ED000FF0096000000000804000000F43C000809
:103EE00000000000000000000000000000000000D2
:083EF0000000000000000000CA
:00000001FF
